:200000000F01030F0200020209040405080703050F01020F02000302090604050805030734
:200020000F01030F0200020209040607080703050F01020F02000302090604050805030710
:200040000F01000F0200000009000001080103010F01000F02000000090000010801030130
:200060000F01000F0200000009000001080103010F01000F02000000090000010801030110
:200080000F0F0F0F0F0F0F0F0F0F0F0F0F0F0F0F0F0F0F0F0F0F0F0F0F0F0F0F0F0F0F0F80
:2000A0000F0F0F0F0F0F0F0F0F0F0F0F0F0F0F0F0F0F0F0F0F0F0F0F0F0F0F0F0F0F0F0F60
:2000C0000F0F0F0F0F0F0F0F0F0F0F0F0F0F0F0F0F0F0F0F0F0F0F0F0F0F0F0F0F0F0F0F40
:2000E0000F0F0F0F0F0F0F0F0F0F0F0F0F0F0F0F0F0F0F0F0F0F0F0F0F0F0F0F0F0F0F0F20
:00000001FF
